:100000000C94280018950000189500001895000021
:10001000189500001895000018950000189500002C
:10002000189500000C948B0D189500001895000091
:10003000189500001895000018950000189500000C
:1000400018950000189500001895000018950000FC
:100050008FE181BD87E181BD8FE58DBFC4E0E8E719
:100060004E2E88E08EBFD8E0F7E05F2EEEEFF7E08F
:10007000A0E6B0E088278D933197E9F783E389B94B
:1000800088E18AB9662481E48ABB81E38BBB8FEB6C
:1000900087BB8FEB88BB88E084BB83E085BB80E0B7
:1000A00081BB8BE382BB80E08FBD81E08EBD8FE1A1
:1000B00081BD87E181BD86E086B980E487B9C398B8
:1000C000C29AD89ADE9AC498C798C598F894A89509
:1000D0007091D10078607093D1007091D1007B7FD6
:1000E0007093D1000027A1EDB0E08C9183FB0EF45A
:1000F00001E041E0041781E009F080E08F930027E0
:10010000A1EDB0E08C9182FB0EF401E041E0041718
:1001100081E009F080E09F91892B882311F40C94F1
:100120009400DC9881E58ABB0E94FA0E7091D100A0
:1001300070627093D100EFEFF1E0A2ECB0E091E0DB
:100140000E9418300091C200003081E009F080E088
:100150008F930091C2000E3F80E010F009F081E023
:100160009F91892B882311F40C94B9008EEB809316
:10017000C2000091C2004AE0040F01BF89E190E093
:100180000E940A2FE6E8F0E60E94512E0027A1ED1A
:10019000B0E08C9183FB0EF401E041E0041711F014
:1001A0000C94DA00E0EAF0E60E94512E0E945D2EE7
:1001B0000C94ED00E2EAF0E60E94512EA1EDB0E0D1
:1001C0008C9182FBA8E6B7E00E942F2F8D938827A1
:1001D0008C930E94492E0E945D2EEAE0F0E0BB273E
:1001E000A0E10E941530073411F40C942D01EBE0CE
:1001F000F0E0A0E1BB278FE08C937BE70E94043006
:10020000ECE0F0E001E010E0A0E1BB277BE70E941A
:100210000630EAE0F0E0A0E1BB2787E48C937BE7BF
:100220000E940430EEE0F0E0A0E1BB2780E08C9378
:100230007BE70E940430E0E1F0E000E010E0A0E1A4
:10024000BB277BE70E940630EFE0F0E0A0E1BB2790
:1002500080E08C937BE70E940430EBE0F0E0ABEBB6
:10026000B0E00E9415300091BB00043618F011F088
:100270000C943C010C943F0184E68093BB0080E722
:1002800097E9ACEBB0E08D939C93ECE0F0E0A6EB4B
:10029000B0E00E941730EEE0F0E0A3ECB0E00E9486
:1002A0001530EFE0F0E0A4ECB0E00E9415300E94C1
:1002B000FE0EE0E1F0E0A3E6B0E00E941730A3E616
:1002C000B0E00E94B82DE0E1F0E0A3E6B0E07BE70B
:1002D0000E940630A6EBB0E00D911C91003050E07A
:1002E000150711F00C947A0181E090E0A6EBB0E0E4
:1002F0008D939C93E4EAF0E60E94512EA8E6B7E0C5
:10030000EBEBF0E00E949D2F0E94492EECEAF0E614
:100310000E94512EA8E6B7E0E6EBF0E00E948E2F97
:100320000E94492EECEAF0E60E94512EA8E6B7E0C2
:10033000E3ECF0E00E949D2F0E94492EECEAF0E6EB
:100340000E94512EA8E6B7E0E4ECF0E00E949D2F59
:100350000E94492EECEAF0E60E94512EA8E6B7E092
:10036000E3E6F0E00E948E2F0E94492E0E945D2E4F
:1003700080E08093D00070916A00777F70936A006C
:1003800080E08093C60086E08093BE008DE080937D
:10039000BF00E9E6F0E0FA93EA930E94501E22962D
:1003A00084E190E00E940A2FDE980E94F62EC49A03
:1003B000EEEAF0E60E94512E0E945D2E88EC90E05D
:1003C0000E940A2FA89581B5886181BD877F81BD74
:1003D000E0E6F0E0FA93EA930E94C6222296A895FE
:1003E00000916000003011F40C9402020E94DA21A6
:1003F000E8EBF0E60E94512E0E945D2E0E94C10E95
:100400000C9407027091D1007F7B7093D100E2ECD5
:10041000F0E60E94512E0E94032284E690E00E94A2
:100420000A2F00916900003018F011F00C941A02A4
:100430000C942102E9E6F0E0FA93EA930E94DF1FB0
:1004400022960027A1EDB0E08C9186FB0EF401E02E
:1004500040E0041711F00C942F020E948D158FEFCD
:100460000E94602E82E390E00E940A2F7894A89563
:1004700081B5886081BDA2EBB0E04D915C91A6EBA7
:10048000B0E00D911C910417150718F011F00C94B1
:100490004B020C94510281E090E0A6EBB0E08D930A
:1004A0009C930027AAE6B0E08C9184FB0EF401E057
:1004B00041E0041781E009F080E08F930027A1ED6F
:1004C000B0E08C9186FB0EF401E040E0041781E07F
:1004D00009F080E09F918923882311F40C94830212
:1004E000E6EBF0E0FA93EA935A924A9280E0A42D68
:1004F000B52D8C9381E00E94A52D0E943B1324967C
:1005000081E00E94A12D80E08093B80080E080937C
:10051000690070916A007F7770936A000027A1EDEF
:10052000B0E08C9186FB0EF401E041E0041711F07D
:100530000C949C020E94FA0EA895ABE6B0E08827C6
:100540008C930027A1EDB0E08C9183FB0EF401E0C9
:1005500041E0041711F00C94B4020E94412EABE666
:10056000B0E08D9388278C93ABE6B0E08C9180301F
:1005700011F00C9487050091D000003081E009F063
:1005800080E08F930027AAE6B0E08C9181FB0EF407
:1005900001E040E0041781E009F080E09F91892BA1
:1005A000882311F40C945704E0E6F0E0FA93EA9300
:1005B0000E94A81E229600916000003018F011F0F1
:1005C0000C94E4020C94570470916A007068709364
:1005D0006A000091D200003011F00C944003409169
:1005E000C60000916000041718F011F00C94FA0294
:1005F0000C944003809160008093C6000027AAE617
:10060000B0E08C9184FB0EF401E040E0041711F09F
:100610000C941A03A0E6B0E08C91A6EBB0E08D93A9
:1006200088278C93ABE6B0E0ECECF0E60E94302E2D
:100630000C9440030027A1EDB0E08C9187FB0EF4F1
:1006400001E041E0041711F00C943A03A0E6B0E099
:100650000D91112741E050E0040F151FA6EBB0E00B
:100660000D931C93ABE6B0E0ECECF0E60E94302E6C
:100670000C944003ABE6B0E0EEECF0E60E94302EC6
:100680000091D200013011F00C94D403009160006D
:10069000013011F00C945203ABE6B0E0EEECF0E662
:1006A0000E94302E00916000023011F00C945E0325
:1006B000ABE6B0E0E0EDF0E60E94302E80E0809303
:1006C000620000916000033081E009F080E08F93C8
:1006D0000091BB00043681E008F080E09F918923FF
:1006E000882311F40C947C03ABEBB0E08C918E5F0B
:1006F0008C9381E08093620000916000043081E07F
:1007000009F080E08F930091BB00023080E010F090
:1007100009F081E09F918923882311F40C949803B8
:10072000ABEBB0E08C9182508C9381E080936200BF
:1007300000916200013011F00C94D4038EB5887FD3
:100740008EBD5A924A928091BB00A42DB52D8C93F8
:1007500081E00E94A52D5A924A928091C000A42D5A
:10076000B52D8C9381E00E94A52D5A924A928091DA
:10077000C100A42DB52D8C9381E00E94A52D0E946F
:10078000B429269683E00E94A12DEBE0F0E0ABEBCC
:10079000B0E07BE70E9404300091D000013011F0FE
:1007A0000C94D40381E08EBD0091D200023011F090
:1007B0000C9457044091C60000916000041718F093
:1007C00011F00C94E5030C94570480916000809321
:1007D000C60000916000013011F00C94FB0381E031
:1007E00090E0A6EBB0E08D939C93ABE6B0E0ECEC30
:1007F000F0E60E94302E00916000023011F00C945F
:100800003F04A2EBB0E00D911C9141E050E0041BCD
:10081000150BA3E6B0E00D931C9302E010E00F93DC
:100820001F93A3E6B0E08D919C918A939A930E94C6
:10083000D12D2296402F512F1F910F91040F151F7C
:10084000A3E6B0E00D931C93A6EBB0E04D915C9154
:10085000A3E6B0E00D911C910417150711F40C9458
:100860000104A3E6B0E08D919C91A6EBB0E08D93DE
:100870009C93ABE6B0E0ECECF0E60E94302E0091E9
:100880006000033011F00C944B04ABE6B0E0EEECEA
:10089000F0E60E94302E00916000043011F00C94BC
:1008A0005704ABE6B0E0E0EDF0E60E94302E002702
:1008B000AAE6B0E08C9184FB0EF401E041E004175D
:1008C00081E009F080E08F930027A1EDB0E08C91EA
:1008D00087FB0EF401E041E0041781E009F080E0BD
:1008E0009F9189238F930091D000013081E009F01E
:1008F00080E09F918923882311F40C94C204A6EB15
:10090000B0E00D911C91013050E0150711F00C94EE
:10091000C204E0E6F0E0FA93EA930E94A81E229651
:1009200000916000003080E010F009F081E08F93CA
:10093000A2EBB0E04D915C91A0E6B0E00D911127E3
:100940000417150781E008F080E09F918923882330
:1009500011F40C94C204A0E6B0E00D91112741E01F
:1009600050E0040F151FA6EBB0E00D931C93ABE60F
:10097000B0E0ECECF0E60E94302E70916A007068F6
:1009800070936A000027AAE6B0E08C9180FB0EF419
:1009900001E040E0041711F00C948705E9E6F0E06F
:1009A000FA93EA930E94501E229600916900043047
:1009B00011F00C94E2040E94920E70916A0070682B
:1009C00070936A0080E080936000009169000230BB
:1009D00081E009F080E08F930091BB00043681E054
:1009E00008F080E09F918923882311F40C9400057E
:1009F000ABEBB0E08C918B5F8C9381E080936000D7
:100A000000916900033081E009F080E08F9300914C
:100A1000BB00053081E009F080E09F9189238823A5
:100A200011F40C94190581E08093BB0081E0809360
:100A3000600000916900033081E009F080E08F934D
:100A40000091BB00053080E010F009F081E09F913B
:100A50008923882311F40C943505ABEBB0E08C911D
:100A600085508C9381E0809360000091600001309C
:100A700011F00C9476058EB5887F8EBD5A924A92FD
:100A80008091BB00A42DB52D8C9381E00E94A52DF3
:100A90005A924A928091C000A42DB52D8C9381E08A
:100AA0000E94A52D5A924A928091C100A42DB52D85
:100AB0008C9381E00E94A52D0E94B429269683E0A4
:100AC0000E94A12DEBE0F0E0ABEBB0E07BE70E94F1
:100AD00004300091D000013011F00C94710581E0D8
:100AE0008EBD70916A00706870936A000091690011
:100AF000013011F00C948705ABE6B0E0EEECF0E6C7
:100B00000E94302E70916A00706870936A00EBE664
:100B1000F0E0ABE6B0E00E94232FABE6B0E08C91B2
:100B2000803081E009F480E08F930091690000300B
:100B300081E009F480E09F91892B8F930091B800A8
:100B4000013081E009F080E09F91892B882311F426
:100B50000C948E020091B800013011F00C94D10574
:100B600080E08093B800ABE6B0E0EEECF0E60E94E7
:100B7000302E0027A1EDB0E08C9187FB0EF401E050
:100B800041E0041711F00C94D10581E090E0A6EB50
:100B9000B0E08D939C93ABE6B0E0ECECF0E60E9405
:100BA000302EABE6B0E0E2EDF0E60E942F3011F01F
:100BB0000C940E0688EC8093BB008EB5887F8EBDAA
:100BC0005A924A928091BB00A42DB52D8C9381E05E
:100BD0000E94A52D5A924A928091C000A42DB52D55
:100BE0008C9381E00E94A52D5A924A928091C10077
:100BF000A42DB52D8C9381E00E94A52D0E94B429CF
:100C0000269683E00E94A12D0091D000013011F0C2
:100C10000C940C0681E08EBD0C94BD0CE4EDF0E666
:100C20000E942F3011F00C944C06EBE0F0E0ABEB9F
:100C3000B0E00E9415308EB5887F8EBD5A924A92E0
:100C40008091BB00A42DB52D8C9381E00E94A52D31
:100C50005A924A928091C000A42DB52D8C9381E0C8
:100C60000E94A52D5A924A928091C100A42DB52DC3
:100C70008C9381E00E94A52D0E94B429269683E0E2
:100C80000E94A12D0091D000013011F00C944A0671
:100C900081E08EBD0C94BD0CE6EDF0E60E942F3095
:100CA00011F00C9494060E943D2EA0E6B0E08C93C7
:100CB00000916000003011F40C9453060E94412E04
:100CC000A0ECB0E08C938EB5887F8EBD5A924A928C
:100CD0008091BB00A42DB52D8C9381E00E94A52DA1
:100CE0005A924A928091C000A42DB52D8C9381E038
:100CF0000E94A52D5A924A928091C100A42DB52D33
:100D00008C9381E00E94A52D0E94B429269683E051
:100D10000E94A12D0091D000013011F00C94920698
:100D200081E08EBD0C94BD0CE8EDF0E60E942F3002
:100D300011F00C94DC060E943D2EA0E6B0E08C93EE
:100D400000916000003011F40C949B060E94412E2B
:100D5000A1ECB0E08C938EB5887F8EBD5A924A92FA
:100D60008091BB00A42DB52D8C9381E00E94A52D10
:100D70005A924A928091C000A42DB52D8C9381E0A7
:100D80000E94A52D5A924A928091C100A42DB52DA2
:100D90008C9381E00E94A52D0E94B429269683E0C1
:100DA0000E94A12D0091D000013011F00C94DA06C0
:100DB00081E08EBD0C94BD0CEAEDF0E60E942F3070
:100DC00011F00C9421075A924A928091BE00A42DF2
:100DD000B52D8C9381E00E94A52D5A924A92809164
:100DE000BF00A42DB52D8C9381E00E94A52D0E94FB
:100DF0007C2A249682E00E94A12D0091C40041E04B
:100E0000042BA0E6B0E00C937091D1007061709358
:100E1000D1008EB5887F8EBDEFE0F0E0A0E6B0E0B7
:100E20007BE70E940430809160008093C4000091B1
:100E3000D000013011F00C941F0781E08EBD0C949E
:100E4000BD0CECEDF0E60E942F3011F00C9464071D
:100E50005A924A9280E0A42DB52D8C9381E00E9495
:100E6000A52D5A924A9280E0A42DB52D8C9381E055
:100E70000E94A52D0E947C2A249682E00E94A12D2A
:100E80000091C4004EEF0423A0E6B0E00C937091F3
:100E9000D1007F7E7093D1008EB5887F8EBDEFE04C
:100EA000F0E0A0E6B0E07BE70E94043080916000B3
:100EB0008093C4000091D000013011F00C946207BF
:100EC00081E08EBD0C94BD0CECECF0E60E942F305E
:100ED00011F00C94D4070091D000013011F00C9463
:100EE00073070E94920EA2EBB0E04D915C91A6EBCD
:100EF000B0E00D911C910417150718F011F00C9437
:100F0000CF070027A1EDB0E08C9186FB0EF401E045
:100F100040E0041711F00C94A007E6EBF0E0FA9320
:100F2000EA935A924A9280E0A42DB52D8C9381E0E9
:100F30000E94A52D0E943B13249681E00E94A12DC2
:100F40000027A1EDB0E08C9186FB0EF401E041E0BA
:100F5000041711F00C94CD070E94C10E0027A1EDDB
:100F6000B0E08C9186FB0EF401E040E0041711F034
:100F70000C94CD07E6EBF0E0FA93EA935A924A928A
:100F800080E0A42DB52D8C9381E00E94A52D0E94B8
:100F90003B13249681E00E94A12D0C94D20780E09F
:100FA0008093C6000C94BD0CEEEDF0E60E942F304D
:100FB00011F00C94E2070E94920E80E08093C6002C
:100FC0000C94BD0CE0EEF0E60E942F3011F00C9472
:100FD0001C080091D000013011F00C941A08002771
:100FE000AAE6B0E08C9183FB0EF401E040E0041728
:100FF00011F00C940C088EB5887F8EBD89B78B7F5D
:1010000089BF70916A00786070936A0084E690E00E
:101010000E940A2F0C941A0870916A00777F7093CF
:101020006A0080E29EE49DBD8CBD81E08EBD89B7E3
:10103000846089BF0C94BD0CEEECF0E60E942F306A
:1010400011F00C94B4080091D000013011F00C9410
:101050002B080E94920EA6EBB0E00E94B82D00274C
:10106000A1EDB0E08C9185FB0EF401E041E00417A6
:1010700011F00C9450080027AAE6B0E08C9184FB94
:101080000EF401E040E0041711F00C944B08A6EBBD
:10109000B0E00E94BE2D7091D1007F7D7093D10091
:1010A000A2EBB0E04D915C91A6EBB0E00D911C91EC
:1010B0000417150718F011F00C9460080C946608DA
:1010C00081E090E0A6EBB0E08D939C930027A1ED2A
:1010D000B0E08C9186FB0EF401E040E0041711F0C3
:1010E0000C948508E6EBF0E0FA93EA935A924A9260
:1010F00080E0A42DB52D8C9381E00E94A52D0E9447
:101100003B13249681E00E94A12D0027A1EDB0E0C1
:101110008C9186FB0EF401E041E0041711F00C9471
:10112000B2080E94C10E0027A1EDB0E08C9186FBB1
:101130000EF401E040E0041711F00C94B208E6EB65
:10114000F0E0FA93EA935A924A9280E0A42DB52DEA
:101150008C9381E00E94A52D0E943B13249681E090
:101160000E94A12D0C94BD0CE0EDF0E60E942F3002
:1011700011F00C942C090091D000013011F00C9466
:10118000C3080E94920EA6EBB0E00D911C910130B5
:1011900050E0150718F011F00C94D0080C94D60804
:1011A000A6EBB0E00E94BE2D0C94DE08A2EBB0E0EE
:1011B0008D919C91A6EBB0E08D939C930027A1EDBF
:1011C000B0E08C9186FB0EF401E040E0041711F0D2
:1011D0000C94FD08E6EBF0E0FA93EA935A924A92F7
:1011E00080E0A42DB52D8C9381E00E94A52D0E9456
:1011F0003B13249681E00E94A12D0027A1EDB0E0D1
:101200008C9186FB0EF401E041E0041711F00C9480
:101210002A090E94C10E0027A1EDB0E08C9186FB47
:101220000EF401E040E0041711F00C942A09E6EBFB
:10123000F0E0FA93EA935A924A9280E0A42DB52DF9
:101240008C9381E00E94A52D0E943B13249681E09F
:101250000E94A12D0C94BD0CE2EEF0E60E942F300E
:1012600011F00C949F09A6EBB0E00E94B82DA2EB00
:10127000B0E04D915C91A6EBB0E00D911C9104178C
:10128000150718F011F00C9447090C944D0981E0F2
:1012900090E0A6EBB0E08D939C938EB5887F8EBDD9
:1012A000A2E7B0E00D911D912D913C91A2E9B0E033
:1012B0000D931D932D933C930027A1EDB0E08C91ED
:1012C00086FB0EF401E040E0041711F00C94950940
:1012D0005A924A92A2E9B0E00D911D912D913C9154
:1012E000A42DB52D0D931D932D933C9384E00E9466
:1012F000A52D5A924A92A6EBB0E08D919C91A42D17
:10130000B52D8D939C9382E00E94A52D5A924A920E
:1013100080E0A42DB52D8C9381E00E94A52D0E9424
:101320009C16269687E00E94A12D0091D0000130E6
:1013300011F00C949D0981E08EBD0C94BD0CE2EA85
:10134000F0E60E942F3011F00C94130AA6EBB0E0E7
:101350000D911C91013050E0150718F011F00C941C
:10136000B3090C94B909A6EBB0E00E94BE2D0C9411
:10137000C109A2EBB0E08D919C91A6EBB0E08D93FA
:101380009C938EB5887F8EBDA2E7B0E00D911D9134
:101390002D913C91A2E9B0E00D931D932D933C93C8
:1013A0000027A1EDB0E08C9186FB0EF401E040E057
:1013B000041711F00C94090A5A924A92A2E9B0E07B
:1013C0000D911D912D913C91A42DB52D0D931D9343
:1013D0002D933C9384E00E94A52D5A924A92A6EB4D
:1013E000B0E08D919C91A42DB52D8D939C9382E0BE
:1013F0000E94A52D5A924A9280E0A42DB52D8C937F
:1014000081E00E94A52D0E949C16269687E00E94EE
:10141000A12D0091D000013011F00C94110A81E04F
:101420008EBD0C94BD0CE4EEF0E60E942F3011F05E
:101430000C94230AECE0F0E0A6EBB0E07BE70E941E
:1014400006300C94BD0CE6EEF0E60E942F3011F051
:101450000C94370A8DE181BD85E181BD0E94920E19
:1014600081B5886081BD0C94330A0C94BD0CABE649
:10147000B0E0E8EEF0E60E942F3081E008F480E072
:101480008F93ABE6B0E0EAEEF0E60E942F3081E009
:1014900010F009F080E09F918923882311F40C94C7
:1014A0000B0B89B78B7F89BF8EB5887F8EBD0E945D
:1014B0003D2EA0E6B0E08C9300916000003011F466
:1014C0000C94570A0E94412EA6EBB0E08D9388271A
:1014D0008C9380E08093D00070916A00777F709346
:1014E0006A00A2EBB0E04D915C91A6EBB0E00D91EB
:1014F0001C910417150780E010F009F081E08F932C
:10150000A6EBB0E00D911C91003050E0150781E092
:1015100009F080E09F91892B882311F40C94AB0A89
:1015200081E090E0A6EBB0E08D939C93E6EBF0E0D9
:10153000FA93EA935A924A9281E0A42DB52D8C93A6
:1015400081E00E94A52D0E943B13249681E00E9419
:10155000A12D0C94090B0027A1EDB0E08C9186FB26
:101560000EF401E040E0041781E009F080E08F9381
:10157000ABE6B0E0E8EEF0E60E942F3081E009F043
:1015800080E09F918923882311F40C94DA0AE6EB1A
:10159000F0E0FA93EA935A924A9281E0A42DB52D95
:1015A0008C9381E00E94A52D0E943B13249681E03C
:1015B0000E94A12D0027A1EDB0E08C9186FB0EF4D6
:1015C00001E040E0041781E009F080E08F93ABE692
:1015D000B0E0EAEEF0E60E942F3081E009F080E012
:1015E0009F918923882311F40C94090BE6EBF0E01A
:1015F000FA93EA935A924A9280E0A42DB52D8C93E7
:1016000081E00E94A52D0E943B13249681E00E9458
:10161000A12D0C94BD0CECEEF0E60E942F3011F0E1
:101620000C945A0B0E943D2EA0E6B0E08C930091E2
:101630006000003011F40C94120B0E94412EABEBB1
:10164000B0E08C938EB5887F8EBD5A924A9280917D
:10165000BB00A42DB52D8C9381E00E94A52D5A923C
:101660004A928091C000A42DB52D8C9381E00E94F8
:10167000A52D5A924A928091C100A42DB52D8C932C
:1016800081E00E94A52D0E94B429269683E00E9445
:10169000A12DEBE0F0E0ABEBB0E07BE70E94043083
:1016A0000091D000013011F00C94580B81E08EBDF8
:1016B0000C94BD0CEEEEF0E60E942F3011F00C946D
:1016C000A80B0E943D2EA0E6B0E08C930091600034
:1016D000003011F40C94610B8091C3008093600082
:1016E0000E94412EA3ECB0E08C93A3ECB0E08C916F
:1016F0008F738C930E94FE0E0091C30040E104237F
:10170000A0E6B0E00C9300916000003111F00C9461
:101710008D0B0E94FA0E0C948F0B0E94FC0EA3EC12
:10172000B0E08C918F7E8C938EB5887F8EBDEEE07D
:10173000F0E0A3ECB0E07BE70E9404300091D00021
:10174000013011F00C94A60B81E08EBD0C94BD0C01
:10175000E0EAF0E60E942F3011F00C940C0C00919E
:10176000C3004FE30423A0E6B0E00C930091D00047
:10177000013011F00C94C10BA0E6B0E08C918058C0
:101780008C930027A1EDB0E08C9186FB0EF401E074
:1017900041E0041711F00C94D20BA0E6B0E08C915C
:1017A000805C8C930027AAE6B0E08C9183FB0EF45A
:1017B00001E041E0041711F00C94E30BA0E6B0E067
:1017C0008C91805E8C938091B600809362008EB580
:1017D000887F8EBD31E0A0E6B0E00E94582E31E057
:1017E000ABEBB0E00E94582E31E0A2E6B0E00E94E0
:1017F000582E8091B2008093620031E0A2E6B0E002
:101800000E94582E0091D000013011F00C940A0C67
:1018100081E08EBD0C94BD0CE0EFF0E60E942F300D
:1018200011F00C948F0CA7EDB0E00D911D912D914E
:101830003C91A3EDB0E04D915D916D917C910E9442
:10184000762FA5E6B0E00D931D932D933D93A5E66D
:10185000B0E00E94A92DA5E6B0E00D911D912D915B
:101860003C9140E052E060E070E00E946A2EA5E604
:10187000B0E00D931D932D933D93A5E6B0E00D913F
:101880001D912D913C91A5ECB0E04C915527662718
:1018900077270E946F2EA5E6B0E04D935D936D9380
:1018A0007D93A5E6B0E00D911D912D913C914AE00C
:1018B00050E060E070E00E946F2EA5E6B0E04D932E
:1018C0005D936D937D9344E150E060E070E0A5E6A8
:1018D000B0E00D911D912D913C910E947B2F0CF455
:1018E00002C00C947D0C00E010E020E030E0A5E6A2
:1018F000B0E00D931D932D933C938EB5887F8EBDE4
:1019000034E0A5E6B0E00E94582E0091D0000130EE
:1019100011F00C948D0C81E08EBD0C94BD0CE2EFA7
:10192000F0E60E942F3011F00C94A70C8EB5887F42
:101930008EBDA4EAB0E00E944B2E0091D000013091
:1019400011F00C94A50C81E08EBD0C94BD0CE4EF5D
:10195000F0E60E942F3011F00C94BD0C8EB5887FFC
:101960008EBD0E9438160091D000013011F00C9409
:10197000BB0C81E08EBD0C94BD0C81E090E00E9418
:101980000A2F0027AAE6B0E08C9187FB0EF401E055
:1019900040E0041718F011F00C94D00C0C94890D51
:1019A00000916900003018F011F00C94D90C0C94DF
:1019B000400DA895E0E6F0E0FA93EA930E94501EED
:1019C000229600916000043011F00C94340D0E94B6
:1019D000920E80E08093C6000E94FC0E85E090E0AD
:1019E0000E940A2F80E080936200E0E6F0E0FA9324
:1019F000EA930E94501E2296A2E6B0E08C918F5F7F
:101A00008C9388E090E00E940A2F009160000030E3
:101A100081E009F080E08F9300916200043680E05D
:101A200010F009F081E09F91892B882311F40C9428
:101A3000F50C00916200043618F011F00C94220DA0
:101A40000C94310D81B5886181BD877F81BDE3E64E
:101A5000F0E0FA93EA930E94B30F229681B5886072
:101A600081BD80E08093600081E090E00E940A2FB9
:101A700000916000003011F00C94D90C0C947F0D93
:101A80000091D200013011F00C947B0D80E090E0C9
:101A9000A3E6B0E08D939C93E0E6F0E0FA93EA933E
:101AA0000E94A81E2296A3E6B0E00E94B82DEF93F4
:101AB000FF93ECE8F1E00E94DE2EFF91EF910091A0
:101AC0006000003081E009F080E08F93A3E6B0E091
:101AD0000D911C91083250E0150780E010F009F0DC
:101AE00081E09F91892B882311F40C944C0D81E0A7
:101AF00090E00E940A2F81E090E00E940A2F00915E
:101B0000D000003011F00C94890D85E090E00E9427
:101B10000A2F0C9489020F921F922F923F924F929C
:101B20005F927F928F929F92AF92BF920F931F937B
:101B30002F933F934F935F936F937F938F939F93D5
:101B4000AF93BF93CF93DF93EF93FF938FB78F93B1
:101B5000F89489B78B7F89BF8EB5887F8EBD5A92E6
:101B60004A9280E092E0A42DB52D8D939C9382E063
:101B70000E94A52D0E941F2D229682E00E94A12D79
:101B80000091DB000A3011F00C94C80D0E94FA0E8F
:101B90000E94FA250091DB000A3011F00C94D50D5B
:101BA0000E94FC0E80E08093DB00ABEDB0E08C91F6
:101BB0008F5F8C93A8950027A1EDB0E08C9186FBF8
:101BC0000EF401E040E0041711F00C94FA0D5A9263
:101BD0004A9280E092E0A42DB52D8D939C9382E0F3
:101BE0000E94A52D0E941F2D229682E00E94A12D09
:101BF0000E94FA25A7EDB0E04D915D916D917C9129
:101C0000A3EDB0E00D911D912D913C910E947B2F91
:101C100080E00CF481E08F930027A1EDB0E08C917F
:101C200086FB0EF401E040E0041781E009F080E05B
:101C30009F918923882311F40C94290E80E49CE958
:101C40009DBD8CBD81E08EBD89B7846089BF0C9439
:101C5000720E80E08093D00070916A00777F70935D
:101C60006A000027A1EDB0E08C9186FB0EF401E044
:101C700040E0041711F00C94460EAAE6B0E08C91F7
:101C800084FBA8EBB0E0882780F98C930091C30017
:101C90004FE70423A1E6B0E00C930E94FC0E80E025
:101CA0008093C6000027A1EDB0E08C9183FB0EF479
:101CB00001E041E0041781E009F080E08F93002704
:101CC000A1EDB0E08C9182FB0EF401E041E004173D
:101CD00081E009F080E09F91892B882311F40C9416
:101CE000720EDC988F918FBFFF91EF91DF91CF91B2
:101CF000BF91AF919F918F917F916F915F914F9124
:101D00003F912F911F910F91BF90AF909F908F9017
:101D10007F905F904F903F902F901F900F9018955D
:101D2000F894FFCF89B78B7F89BF8EB5887F8EBD32
:101D300080E08093D00070916A00777F70936A0092
:101D40000027A1EDB0E08C9183FB0EF401E041E0AF
:101D5000041781E009F080E08F930027A1EDB0E047
:101D60008C9182FB0EF401E041E0041781E009F060
:101D700080E09F91892B882311F40C94C00EDC988D
:101D80000895DE9A6E98C498C598C7980E94FC0E74
:101D9000E2E0F0E00E94642EDE98C49A0E94F62EE3
:101DA00084E690E00E940A2FA8957091D1007F7B75
:101DB0007093D100E0E6F0E0FA93EA930E94C62225
:101DC000229600916000003011F40C94F70E70918F
:101DD000D10070647093D10084E690E00E940A2FD5
:101DE000DE9A6E98C498C598C7980C94F90E0E9414
:101DF0008D150895AB980895AB9A089581E00E94DF
:101E0000192F70916A007F7E70936A000091C30061
:101E100041E00423A881B9810C93A881B9810C9178
:101E2000003011F40C94190F70916A007061709376
:101E30006A007091D1007F777093D1000091C30048
:101E400042E00423A881B9810C93A881B9810C9147
:101E5000003011F40C94310F7091D10070687093C0
:101E6000D10070916A007E7F70936A000091C30078
:101E700044E00423A881B9810C93A881B9810C9115
:101E8000003011F40C94490F70916A0071607093E6
:101E90006A0070916A007D7F70936A000091C300B0
:101EA00048E00423A881B9810C93A881B9810C91E1
:101EB000003011F40C94610F70916A00726070939D
:101EC0006A0070916A007F7D70936A000091C30080
:101ED00040E20423A881B9810C93A881B9810C91B7
:101EE000003011F40C94790F70916A007062709355
:101EF0006A007091D1007F7E7093D1000091C40080
:101F000041E00423A881B9810C93A881B9810C9187
:101F1000003011F40C94910F7091D10070617093A6
:101F2000D1000091C40046E00423A881B9810C933C
:101F3000A881B9810C9142E00E941F300C93A881C6
:101F4000B9818C918093D2000091D200033011F0BE
:101F50000C94AD0F82E08093D20081E0481A88276C
:101F6000580A2296089582E00E94192F81E00E946B
:101F7000192F81E00E94192F80E0AA81BB818C93E8
:101F800083E4ACE9B0E08C938FE4ADE9B0E08C93EE
:101F90008EE4AEE9B0E08C9386E4AFE9B0E08C93D8
:101FA00089E4A0EAB0E08C93AAE6B0E08C9185FBCE
:101FB000A881B981882780F98C9370916A0070623A
:101FC00070936A00A2E7B0E00D911D912D913C91B4
:101FD000A2E9B0E00D931D932D933C935A924A923F
:101FE000A2E9B0E00D911D912D913C91A42DB52D4C
:101FF0000D931D932D933C9384E00E94A52D5A923E
:102000004A9280E090E0A42DB52D8D939C9382E0C0
:102010000E94A52D5A924A9281E0A42DB52D8C9351
:1020200081E00E94A52D0E949C16269687E00E94C2
:10203000A12D8FE00E94192FE4EAF0E006E0A881CC
:10204000B9810E94F62FA881B981E6EFF0E60E94DF
:102050002F300FB68FE0481A8827580A22960FBEF5
:1020600081E009F080E08F9300918D00003181E0E4
:1020700009F080E09F918923882311F40C948E103D
:1020800081E0AA81BB818C93A2E9B0E00D911D9102
:102090002D913C91A2E7B0E00D931D932D933C93BD
:1020A00070916A007F7D70936A005A924A92A2E909
:1020B000B0E00D911D912D913C91A42DB52D0D9366
:1020C0001D932D933C9384E00E94A52D5A924A9231
:1020D00080E090E0A42DB52D8D939C9382E00E942A
:1020E000A52D5A924A9280E0A42DB52D8C9381E0C3
:1020F0000E94A52D0E949C16269687E00E94A12D85
:10210000A2E9B0E00D911D912D913C91A2E7B0E0C4
:102110000D931D932D933C930E94E810A881B981E3
:102120008C9180FBAAE6B0E08C9185F98C93A6E7B0
:10213000B0E00D911D912D913C91A2E7B0E00D937F
:102140001D932D933C93A2E7B0E00D911D912D912D
:102150003C91A2E9B0E00D931D932D933C935A92CC
:102160004A92A2E9B0E00D911D912D913C91A42DD0
:10217000B52D0D931D932D933C9384E00E94A52DC6
:102180005A924A9280E090E0A42DB52D8D939C93B5
:1021900082E00E94A52D5A924A9280E0A42DB52D8E
:1021A0008C9381E00E94A52D0E949C16269687E0C4
:1021B0000E94A12DAA81BB818C91AE81BF818D939C
:1021C00088278C9384E0481A8827580A2696089511
:1021D00082E00E94192F81E00E94192F81E00E9465
:1021E000192F789481E090E0AC81BD818D939C9310
:1021F000EA81FB81FA93EA93EE81FF81FA93EA93F5
:102200000E94FE122496AA81BB810C91013011F02C
:102210000C94151182E090E0AC81BD818D939C936C
:1022200081E08093C3000C943111023011F00C94C2
:10223000241183E090E0AC81BD818D939C9380E07C
:102240008093C3000C943111033011F00C943111C0
:1022500084E090E0AC81BD818D939C9383E080937A
:10226000C300EEE0F0E0A3ECB0E07BE70E940430B6
:10227000EC81FD81FA93EA935A924A9280E0A42D70
:10228000B52D8C9381E00E94A52D0E943B132496CE
:1022900081E00E94A12D0091D000003011F00C943B
:1022A0004B1188EC90E00E940A2F85E090E0AC8111
:1022B000BD818D939C93EA81FB81FA93EA93EE8131
:1022C000FF81FA93EA930E94FE122496EEE0F0E07A
:1022D000A3ECB0E00E941530AA81BB810C910330C1
:1022E00011F00C9475110C941212AA81BB810C91FF
:1022F000013011F00C948311A3ECB0E08C91886054
:102300008C930C948C11023011F00C948C11A3EC72
:10231000B0E08C91877F8C93EEE0F0E0A3ECB0E02E
:102320007BE70E94043088EC90E00E940A2F86E050
:1023300090E0AC81BD818D939C93EA81FB81FA93FF
:10234000EA93EE81FF81FA93EA930E94FE122496AB
:10235000AA81BB810C91033011F00C94B1110C9443
:102360001212EEE0F0E0A3ECB0E00E941530AA817A
:10237000BB810C91013011F00C94C511A3ECB0E0BD
:102380008C9184608C930C94CE11023011F00C94DB
:10239000CE11A3ECB0E08C918B7F8C93EEE0F0E05B
:1023A000A3ECB0E07BE70E94043088EC90E00E9450
:1023B0000A2F87E090E0AC81BD818D939C93EA81E8
:1023C000FB81FA93EA93EE81FF81FA93EA930E94EC
:1023D000FE122496EEE0F0E0A3ECB0E00E9415308F
:1023E000AA81BB810C91013011F00C94FE11A3EC79
:1023F000B0E08C9180628C930C940712023011F043
:102400000C940712A3ECB0E08C918F7D8C93EEE0DE
:10241000F0E0A3ECB0E07BE70E94043088EC90E0B1
:102420000E940A2F88E090E0AC81BD818D939C933F
:10243000EC81FD81FA93EA930E94DC1222960091CE
:10244000C30043E00423A881B9810C93A881B9811A
:102450000C91003011F00C94351283E090E0AC81C7
:10246000BD818D939C930C944B12013011F00C9410
:10247000411282E090E0AC81BD818D939C930C94DD
:102480004B12033011F00C944B1284E090E0AC81BD
:10249000BD818D939C93EC81FD81FA93EA930E9418
:1024A000DC1222960091C30048E00423A881B98180
:1024B0000C93A881B9810C91003011F00C94681232
:1024C0008AE090E0AC81BD818D939C930C94721254
:1024D000083011F00C94721289E090E0AC81BD815B
:1024E0008D939C93EC81FD81FA93EA930E94DC1218
:1024F00022960091C30044E00423A881B9810C9383
:10250000A881B9810C91003011F00C948F128BE0EE
:1025100090E0AC81BD818D939C930C949912043012
:1025200011F00C9499128CE090E0AC81BD818D93F8
:102530009C93EC81FD81FA93EA930E94DC1222962F
:102540000091C30040E20423A881B9810C93A881C3
:10255000B9810C91003011F00C94B6128DE090E02E
:10256000AC81BD818D939C930C94C012003211F00C
:102570000C94C0128EE090E0AC81BD818D939C9351
:10258000EC81FD81FA93EA930E94DC1222968FE09F
:1025900090E0AC81BD818D939C93EC81FD81FA9399
:1025A000EA930E94DC1222960E94FE0E84E0481AF2
:1025B0008827580A26960895E881F981FA93EA93C4
:1025C0005A924A9280E0A42DB52D8C9381E00E940E
:1025D000A52D0E943B13249681E00E94A12D82E349
:1025E00090E00E940A2F0091D000003011F00C946E
:1025F000F31282E390E00E940A2F089581E00E9486
:10260000192FEA81FB81FA93EA935A924A9280E069
:10261000A42DB52D8C9381E00E94A52D0E943B1323
:10262000249681E00E94A12D84E690E00E940A2F6A
:10263000E881F981FA93EA930E94501E2296A881BC
:10264000B9810C91003018F011F00C9429130C94FE
:1026500018130E94920E84E190E00E940A2FA88134
:10266000B9818C91AC81BD818C9381E0481A882717
:10267000580A2296089582E00E94192F81E00E9454
:10268000192F8EB5887F8EBD70916A00777F709309
:102690006A00A2E7B0E00D911D912D913C91A2E955
:1026A000B0E00D931D932D933C935A924A92A2E968
:1026B000B0E00D911D912D913C91A42DB52D0D9360
:1026C0001D932D933C9384E00E94A52D5A924A922B
:1026D000AA85BB858D919C91A42DB52D8D939C933E
:1026E00082E00E94A52D5A924A9280E0A42DB52D39
:1026F0008C9381E00E94A52D0E949C16269687E06F
:102700000E94A12D40E050E060E070E0AEE8B0E053
:102710000D911D912D913C910E947B2F11F00C94F5
:1027200093130C9487150E9468295A924A928091BB
:10273000BB00A42DB52D8C9381E00E94A52D5A924B
:102740004A928091C000A42DB52D8C9381E00E9407
:10275000A52D5A924A928091C100A42DB52D8C933B
:1027600081E00E94A52D0E94B429269683E00E9454
:10277000A12D5A924A92ACEBB0E08D919C91A42D80
:10278000B52D8D939C9382E00E94A52D0E94BB2ABB
:10279000229682E00E94A12D0027A1EDB0E08C914D
:1027A00084FB0EF401E041E0041711F00C94F213E5
:1027B0005A924A928091BE00A42DB52D8C9381E04F
:1027C0000E94A52D5A924A928091BF00A42DB52D4A
:1027D0008C9381E00E94A52D0E947C2A249682E0A1
:1027E0000E94A12DA2E9B0E00D911D912D913C9187
:1027F000A3EDB0E00D931D932D933C93A2E9B0E0BF
:102800000D911D912D913C91AEE8B0E04D915D91FF
:102810006D917C910E94712FA7EDB0E00D931D93F7
:102820002D933D9380E0A881B9818C930E94FA2575
:1028300081E090E0AA81BB818D939C93AA81BB81AA
:102840000D911C910F3F51E0150718F011F00C94F9
:102850005814AA81BB81AD90BC90ABEDB0E0AA0D3D
:10286000BB1D0C910F3F81E009F080E08F93AA819E
:10287000BB81AD90BC90ACEDB0E0AA0DBB1D0C913E
:102880000F3E80E010F009F081E09F9189238823BA
:1028900011F40C94511481E0A881B9818C930C94AB
:1028A0005814AA81BB810E94B82D11F00C941E14FB
:1028B000A881B9810C91013011F00C941614AA81F1
:1028C000BB81AD90BC90ADEDB0E0AA0DBB1D8C916D
:1028D000AA81BB818D9388278C93AA81BB810D919E
:1028E0001C9140E150E00E94EA2DAA81BB814D93EA
:1028F0005C9380E18093C500AA81BB810D911C91FE
:10290000013050E0150711F00C948B1484E0809393
:10291000C5000C941815023050E0150711F00C9406
:10292000961485E08093C5000C941815033050E090
:10293000150711F00C94A11486E08093C5000C9447
:102940001815043050E0150711F00C94AC1487E012
:102950008093C5000C941815053050E0150711F050
:102960000C94B71488E08093C5000C9418150630B9
:1029700050E0150711F00C94C2148AE08093C50052
:102980000C941815073050E0150711F00C94CD1475
:102990008CE08093C5000C941815083050E01507A2
:1029A00011F00C94D8148EE08093C5000C94181587
:1029B000093050E0150711F00C94E31480E1809386
:1029C000C5000C9418150A3050E0150711F00C944E
:1029D000EE1484E18093C5000C9418150B3050E080
:1029E000150711F00C94F91488E18093C5000C943C
:1029F00018150C3050E0150711F00C9404158CE1FB
:102A00008093C5000C9418150D3050E0150711F097
:102A10000C940F1580E28093C5000C9418150E30AD
:102A200050E0150711F00C94181588E28093C5004A
:102A3000AEE8B0E00D911D912D913C9140E052E047
:102A400060E070E00E946A2EA5E6B0E00D931D9351
:102A50002D933D93A5E6B0E00D911D912D913C91F4
:102A6000A5ECB0E04C915527662777270E946F2E82
:102A7000A5E6B0E04D935D936D937D93A5E6B0E040
:102A80000D911D912D913C9148EE53E060E070E076
:102A90000E946F2EA5E6B0E04D935D936D937D93FC
:102AA000AC81BD810C91003011F00C94871581E050
:102AB0008093D00088EC9FEA9DBD8CBD89B784606F
:102AC00089BF81E08EBD0027A1EDB0E08C9183FB32
:102AD0000EF401E041E0041781E009F080E08F93FB
:102AE0000027A1EDB0E08C9182FB0EF401E041E003
:102AF000041781E009F080E09F91892B882311F46D
:102B00000C948315DC9A85E090E00E940A2F83E004
:102B1000481A8827580A24960895A895A2E7B0E095
:102B20000D911D912D913C91A6E7B0E00D931D9361
:102B30002D933C93A2E7B0E00D911D912D913C9116
:102B4000A2E9B0E00D931D932D933C935A924A92C3
:102B5000A2E9B0E00D911D912D913C91A42DB52DD0
:102B60000D931D932D933C9384E00E94A52D5A92C2
:102B70004A9280E090E0A42DB52D8D939C9382E045
:102B80000E94A52D5A924A9280E0A42DB52D8C93D7
:102B900081E00E94A52D0E949C16269687E00E9447
:102BA000A12DA895A2EBB0E00D911C91013050E051
:102BB000150710F00C9403165A924A9281E0A42D46
:102BC000B52D8C9381E00E94A52D0E94152B229695
:102BD00081E00E94A12D8CE291E00E940A2F5A927E
:102BE0004A9280E0A42DB52D8C9381E00E94A52D02
:102BF0000E94152B229681E00E94A12D7091D10098
:102C000070647093D100A895A2E7B0E00D911D917A
:102C10002D913C91A2E9B0E00D931D932D933C932F
:102C2000A6EBB0E00D911C91003050E0150781E05B
:102C300009F080E08F93A2EBB0E04D915C91A6EBA0
:102C4000B0E00D911C910417150780E010F009F019
:102C500081E09F91892B882311F40C94351681E033
:102C600090E0A6EBB0E08D939C930E94FC0E08953B
:102C700084E00E94192FA3EDB0E00D911D912D91DC
:102C80003C91A881B9810D931D932D933C93A2E7AC
:102C9000B0E00D911D912D913C91A2E9B0E00D9312
:102CA0001D932D933C935A924A92A2E9B0E00D9164
:102CB0001D912D913C91A42DB52D0D931D932D9318
:102CC0003C9384E00E94A52D5A924A928FE19EE4A3
:102CD000A42DB52D8D939C9382E00E94A52D5A9230
:102CE0004A9280E0A42DB52D8C9381E00E94A52D01
:102CF0000E949C16269687E00E94A12DA2E7B0E0D4
:102D00000D911D912D913C91A2E9B0E00D931D9381
:102D10002D933C93A881B9810D911D912D913C91EA
:102D2000A3EDB0E00D931D932D933C9384E0481ADE
:102D30008827580A2296089581E00E94192F81E081
:102D40000E94192F81E00E94192F80E090E0A4EBEF
:102D5000B0E08D939C9370916A007F7B70936A00C2
:102D600000E010E020E030E0AEE8B0E00D931D930D
:102D70002D933C930027AAE6B0E08C9185FB0EF4DE
:102D800001E041E0041781E009F080E08F93A8851D
:102D9000B9850D911C91003050E0150781E009F4D0
:102DA00080E09F9189238F93AE81BF810C91003089
:102DB00081E009F080E09F918923882311F40C942D
:102DC0003C17A6E9B0E0E885F9850E948E2FE6E978
:102DD000F0E0A8E6B7E00E94EA2FE8E6F7E0A6E90F
:102DE000B0E01127222704E033270E94332F81E42B
:102DF000AC81BD818C93AC81BD818C9180939C0012
:102E000081E0E6E9F0E001E00A93ABE6B0E00E9481
:102E1000EF2FABE6B0E08C91ADE9B0E08C9382E0AF
:102E2000E6E9F0E001E00A93ABE6B0E00E94EF2FA4
:102E3000ABE6B0E08C91AEE9B0E08C9383E0E6E9DC
:102E4000F0E001E00A93ABE6B0E00E94EF2FABE6C2
:102E5000B0E08C91AFE9B0E08C9384E0E6E9F0E07B
:102E600001E00A93ABE6B0E00E94EF2FABE6B0E0E2
:102E70008C91A0EAB0E08C9389B78B7F89BF8EB527
:102E8000887F8EBD81B5886181BD877F81BDACECB7
:102E9000B0E00D911D912D913C91A8ECB0E00D9307
:102EA0001D932D933C93A6E7B0E04D915D916D91FC
:102EB0007C91A2E7B0E00D911D912D913C910E9473
:102EC0007B2F11F00C946E1702E010E020E030E050
:102ED000A8ECB0E00D931D932D933C9380E0A88166
:102EE000B9818C93EA81FB81FA93EA935A924A92D0
:102EF000AE85BF850D911D912D913C91A42DB52DD1
:102F00000D931D932D933C9384E00E94A52D0E9468
:102F1000F127249684E00E94A12DAA81BB810C9107
:102F20000E3F11F40C94A0177091D100706470934F
:102F3000D10070916A00706470936A000C94B317AA
:102F40005A924A92AA85BB858D919C91A42DB52D4C
:102F50008D939C9382E00E94A52D0E94B418229626
:102F600082E00E94A12DA881B9818C918F5F8C9302
:102F700040916F00A881B9810C91041781E009F09C
:102F800080E08F930027AAE6B0E08C9186FB0EF4D8
:102F900001E041E0041781E009F480E09F9189237A
:102FA000882311F40C94691800917E000B3011F005
:102FB0000C941618E8ECF0E0FA93EA935A924A92CD
:102FC000A8ECB0E00D911D912D913C91A42DB52D53
:102FD0000D931D932D933C9384E00E94A52D0E9498
:102FE000F41C249684E00E94A12DEA85FB85FA93C7
:102FF000EA935A924A92A8ECB0E00D911D912D915E
:103000003C91A42DB52D0D931D932D933C9384E0FD
:103010000E94A52D0E948A1C249684E00E94A12D66
:1030200080E0A881B9818C930C946718A6E7B0E082
:103030004D915D916D917C91A2E7B0E00D911D9154
:103040002D913C910E947B2F11F00C942D18AA8594
:10305000BB850E94A92D0C946718E8ECF0E0FA9368
:10306000EA935A924A92A8ECB0E00D911D912D91ED
:103070003C91A42DB52D0D931D932D933C9384E08D
:103080000E94A52D0E94F41C249684E00E94A12D8C
:10309000EA85FB85FA93EA935A924A92A8ECB0E04B
:1030A0000D911D912D913C91A42DB52D0D931D9346
:1030B0002D933C9384E00E94A52D0E948A1C2496A7
:1030C00084E00E94A12D80E0A881B9818C930C94AA
:1030D0006D18AA85BB850E94A92D0027AAE6B0E03D
:1030E0008C9186FB0EF401E041E0041711F00C9482
:1030F0007217C49AA885B9850D911C91003050E0D3
:10310000150711F00C948C18A4EBB0E08D919C91F4
:10311000A2EBB0E08D939C930091D000013081E050
:1031200009F080E08F930027A1EDB0E08C9186FB41
:103130000EF401E040E0041781E009F080E09F9187
:103140008923882311F40C94AE1880E593EC9DBD7F
:103150008CBD81E08EBD89B7846089BF83E0481A49
:103160008827580A2696089584E00E94192F84E043
:103170000E94192F81E00E94192F81E00E94192FCF
:1031800081E00E94192F81E00E94192F80E0AE811A
:10319000BF818C93AE81BF810C910F3018F011F07C
:1031A0000C94971A81E0AC81BD818C93AC81BD8178
:1031B0000C910C3018F011F00C94F6188FEF0E945F
:1031C000FD2E0E94FF2E0E94FE2EAC81BD81AD908F
:1031D000BB24A0E8B0E0AA0DBB1D8C93AC81BD81DF
:1031E0008C918F5F8C9311F00C94D6188DE0AC818C
:1031F000BD818C93AC81BD810C91043118F011F02C
:103200000C9414198FEF0E94FD2E0E94FF2E0E9435
:10321000FE2EA881B9818C93AC81BD818C918F5F8A
:103220008C9311F00C94FA18EA85FB85FA93EA93D3
:10323000EA85FB85FA93EA930E941F1B24960027D8
:10324000AAE6B0E08C9186FB0EF401E041E00417A1
:1032500011F00C942D190C948F1A80E0AA81BB8177
:103260008C9300918C00003281E009F080E08F9314
:1032700000918C00003181E009F080E09F91892B62
:10328000882311F40C94481981E0AA81BB818C93A6
:1032900000918100003081E009F480E08F9300917B
:1032A0008100053E81E009F480E09F9189238F939E
:1032B000AA81BB810C91013081E009F080E09F91EF
:1032C0008923882311F40C94841A00918C00003215
:1032D00011F00C946F19A4EBB0E00E94B82D0027F8
:1032E000AAE6B0E08C9185FB0EF401E040E0041703
:1032F00011F00C94A41981E0AC81BD818C93AC8554
:10330000BD854D915C91A4EBB0E00D911C9104172B
:10331000150781E009F080E08F93A4EBB0E00D91F8
:103320001C91003050E0150780E010F009F081E0BA
:103330009F918923882311F40C94A21980E0AC8119
:10334000BD818C930C94D81980E0AC81BD818C93A5
:1033500081E0A881B9818C93A881B9810C91053055
:1033600018F011F00C94D819A881B981AD90BB2444
:10337000ABE9B0E0AA0DBB1D4C91A881B981AD901D
:10338000BB24A0E8B0E0AA0DBB1D0C91041711F4FA
:103390000C94D01981E0AC81BD818C930C94D81928
:1033A000A881B9818C918F5F8C9311F00C94AC192A
:1033B000AC81BD810C91003081E009F080E08F93F9
:1033C000AC85BD850D911C910F315EE4150781E040
:1033D00009F080E09F91892B882311F40C94841AC2
:1033E0000E94B11AA885B9850D911D912D913C912E
:1033F00040E052E060E070E00E946F2EAEE8B0E086
:103400004D935D936D937D93E2E9F0E0FA93EA9337
:103410005A924A92AE85BF850D911D912D913C9196
:10342000A42DB52D0D931D932D933C9384E00E9404
:10343000A52D0E948A1C249684E00E94A12D8091D3
:103440008C0080938D00AC85BD850D911C910F3152
:103450005EE4150711F00C94551AA8E6B7E0E4EB0A
:10346000F0E00E948E2F0E94492EEEEFF0E60E94BF
:10347000512EA4EAB0E00E944B2EEEEFF0E60E943F
:10348000512E00918C00003111F00C944B1AE0E0A9
:10349000F1E60E94512EA8E6B7E0E885F9850E9482
:1034A000912F0E94492E0E945D2EAC81BD810C910E
:1034B000003011F00C94841A70916A00706470935B
:1034C0006A0000918D00003181E009F080E08F9367
:1034D000AC85BD850D911C910F315EE4150781E02F
:1034E00009F480E09F918923882311F40C94841AB5
:1034F000AA85BB850D911D912D913C91ACECB0E05E
:103500000D931D932D933C9300918100003011F099
:103510000C948F1A70916A00706470936A00AE8187
:10352000BF818C918F5F8C9311F00C94CA188FEF30
:103530000E94FD2E0E94FF2E0E94FE2EA0E6B0E00B
:103540008C938FEF0E94FD2E0E94FF2E0E94FE2E74
:10355000A0E6B0E08C938CE0481A8827580A2C9695
:10356000089581E00E94192FA4EAB0E088278C9387
:1035700081E0A881B9818C93A881B9810C91083030
:1035800018F011F00C94EB1AA881B981AD90BB240E
:10359000A0E8B0E0AA0DBB1D0C91003211F40C9410
:1035A000E31AA881B981AD90BB24A0E8B0E0AA0DD0
:1035B000BB1D8C91A4EAB0E08F930E94362E8F91B0
:1035C0008D9388278C93A881B9818C918F5F8C9380
:1035D00011F00C94BC1AA4EAB0E00E94362EE4E08C
:1035E000F1E60E94302E89E0A881B9818C93A881F0
:1035F000B9810C910B3018F011F00C94191BA881B3
:10360000B981AD90BB24A0E8B0E0AA0DBB1D8C91A0
:10361000A4EAB0E08F930E94362E8F918D93882775
:103620008C93A881B9818C918F5F8C9311F00C944D
:10363000F71A81E0481A8827580A2296089581E0EF
:103640000E94192F81E00E94192F84E00E94192FF7
:103650008FEF0E94FD2E0E94FF2E0E94FE2EAC8155
:10366000BD818C938FEF0E94FD2E0E94FF2E0E9441
:10367000FE2EAA81BB818C93AA81BB810C9111275C
:103680002227332740E051E060E070E00E946A2E7C
:10369000A885B9850D931D932D933D93A885B98574
:1036A0000D911D912D913C91AC81BD814C9155277F
:1036B000662777270E94712FA885B9850D931D93E2
:1036C0002D933D93A885B9850D911D912D913C9128
:1036D00040E050E061E070E00E946A2EA881B9816C
:1036E0000D931D932D933D938FEF0E94FD2E0E940D
:1036F000FF2E0E94FE2EAC81BD818C938FEF0E9425
:10370000FD2E0E94FF2E0E94FE2EAC81BD818C9367
:103710008FEF0E94FD2E0E94FF2E0E94FE2EAC8194
:10372000BD818C938FEF0E94FD2E0E94FF2E0E9480
:10373000FE2EAC81BD818C938FEF0E94FD2E0E94E6
:10374000FF2E0E94FE2EAC81BD818C938FEF0E94D4
:10375000FD2E0E94FF2E0E94FE2EAA81BB818C931B
:10376000AA81BB810C9111272227332740E051E029
:1037700060E070E00E946A2EA885B9850D931D93C4
:103780002D933D93A885B9850D911D912D913C9167
:10379000AC81BD814C915527662777270E94712FF8
:1037A000A885B9850D931D932D933D93A885B98563
:1037B0000D911D912D913C91A881B9814D915D9103
:1037C0006D917C910E94712FA885B9850D931D93F1
:1037D0002D933D938FEF0E94FD2E0E94FF2E0E949D
:1037E000FE2EAC81BD818C938FEF0E94FD2E0E9436
:1037F000FF2E0E94FE2EAA81BB818C93AA81BB81E1
:103800000C9111272227332740E051E060E070E05F
:103810000E946A2EA881B9810D931D932D933D932B
:10382000A881B9810D911D912D913C91AC81BD81F3
:103830004C915527662777270E94712FA881B9815F
:103840000D931D932D933D938FEF0E94FD2E0E94AB
:10385000FF2E0E94FE2EAC81BD818C938FEF0E94C3
:10386000FD2E0E94FF2E0E94FE2EAA81BB818C930A
:10387000AA81BB810C9111272227332740E051E018
:1038800060E070E00E946A2EAE81BF810D931D93AF
:103890002D933D93AE81BF810D911D912D913C9152
:1038A000AC81BD814C915527662777270E94712FE7
:1038B000AE81BF810D931D932D933D93AE81BF814A
:1038C0000D911D912D913C9140E050E061E070E040
:1038D0000E946A2EAE81BF810D931D932D933D935F
:1038E000AE81BF810D911D912D913C91A881B9812F
:1038F0004D915D916D917C910E94712FAE81BF8140
:103900000D931D932D933D9386E0481A8827580AFE
:103910002696089584E00E94192F84E00E94192FB2
:10392000AC81BD810D911D912D913C9142E050E003
:1039300060E070E00E94762FA881B9810D931D93FD
:103940002D933D93AFE6B0E00C911127222733274A
:10395000A881B9814D915D916D917C910E946A2EF3
:10396000AA81BB810D931D932D933D93AA81BB81A9
:103970000D911D912D913C91A6E7B0E04D915D9187
:103980006D917C910E94712FAA81BB810D931D9333
:103990002D933D9300917E000B3011F40C94E21CAA
:1039A000AA81BB810D911D912D913C9140E250E087
:1039B00060E070E00E94712FAA81BB810D931D937E
:1039C0002D933D93AA81BB810D911D912D913C9129
:1039D000AE81BF810D931D932D933C9388E0481ACF
:1039E0008827580A2496089584E00E94192F82E0BF
:1039F0000E94192F00917E000B3011F00C94381D9D
:103A0000AC81BD810D911D912D913C9140E850E01C
:103A100060E070E00E946F2EA3EDB0E04D935D93E7
:103A20006D937D93AC81BD810D911C9140E850E078
:103A30000E940A2EA881B9810D931C93A881B98197
:103A40000D911C9144E050E00E94242EA881B98180
:103A50000D931C93A881B9810D911C9144E050E015
:103A6000040F151FA881B9810D931C930C946E1D32
:103A7000AC81BD810D911D912D913C9140E051E0B3
:103A800060E070E00E946F2EA3EDB0E04D935D9377
:103A90006D937D93AC81BD810D911C9140E051E00F
:103AA0000E940A2EA881B9810D931C93A881B98127
:103AB0000D911C9142E050E00E94242EA881B98112
:103AC0000D931C93A881B9810D911C9142E050E0A7
:103AD000040F151FA881B9810D931C93A3EDB0E0CD
:103AE0000D911D912D913C91AAE7B0E04D915D9112
:103AF0006D917C910E94712FA3EDB0E00D931D9309
:103B00002D933D93A3EDB0E00D911D912D913C912E
:103B1000ADE6B0E04D915C91662777270E94712F4A
:103B2000A3EDB0E00D931D932D933D930E94FA25D4
:103B3000A881B981AD90BC90ABEDB0E0AA0DBB1DE2
:103B40008C91AA81BB818D9388278D938D938C93C3
:103B5000A881B9810E94BE2DAA81BB810D911D91C2
:103B60002D913C9140E051E060E070E00E946A2EAF
:103B7000AA81BB810D931D932D933D93AA81BB8197
:103B80000D911D912D913C91A881B981AD90BC9072
:103B9000ABEDB0E0AA0DBB1D4C91552766277727EA
:103BA0000E94712FAA81BB810D931D932D933D938C
:103BB00000917E000B3011F00C943E1EA881B9815B
:103BC0000E94BE2DAA81BB810D911D912D913C912A
:103BD00040E051E060E070E00E946A2EAA81BB8163
:103BE0000D931D932D933D93AA81BB810D911D9142
:103BF0002D913C91A881B981AD90BC90ABEDB0E026
:103C0000AA0DBB1D4C915527662777270E94712F5F
:103C1000AA81BB810D931D932D933D93A881B981FA
:103C20000E94BE2DAA81BB810D911D912D913C91C9
:103C300040E051E060E070E00E946A2EAA81BB8102
:103C40000D931D932D933D93AA81BB810D911D91E1
:103C50002D913C91A881B981AD90BC90ABEDB0E0C5
:103C6000AA0DBB1D4C915527662777270E94712FFF
:103C7000AA81BB810D931D932D933D93AA81BB8196
:103C80000D911D912D913C91AE81BF810D931D939E
:103C90002D933C9386E0481A8827580A2496089565
:103CA00080E0A881B9818C930027BB27A0E38C9189
:103CB00083FB0EF401E040E0041711F00C94641E45
:103CC00082E0A881B9818C930027BB27A0E38C9167
:103CD00084FB0EF401E040E0041711F00C94741E14
:103CE00081E0A881B9818C930027BB27A3E38C9145
:103CF00081FB0EF401E040E0041711F00C94841EE7
:103D000083E0A881B9818C930027BB27A3E38C9122
:103D100081FB0EF401E040E0041781E009F080E04F
:103D20008F930027BB27A0E38C9183FB0EF401E067
:103D300040E0041781E009F080E09F918923882307
:103D400011F40C94A71E84E0A881B9818C93089586
:103D500081E00E94192F81E00E94192F82E00E94C9
:103D6000192F0027A1EDB0E08C9183FB0EF401E048
:103D700041E0041711F00C94D31E80E0AC81BD81AA
:103D80008C930027BB27A9E38C9185FB0EF401E0FF
:103D900040E0041711F00C94D11E81E0AC81BD818C
:103DA0008C930C94D31F5398549880E081BB909AC5
:103DB000919AEF93FF93E0EFF1E00E94DE2EFF91E6
:103DC000EF9180E0AC81BD818C930027BB27A0E3FD
:103DD0008C9180FB0EF401E040E0041711F00C948C
:103DE000F51E81E0AC81BD818C930027BB27A0E349
:103DF0008C9181FB0EF401E040E0041711F00C946B
:103E0000061FAC81BD818C918E5F8C930027BB27F0
:103E1000A9E38C9185FB0EF401E040E0041711F05A
:103E20000C94171FAC81BD818C918C5F8C93002703
:103E3000BB27A9E38C9184FB0EF401E040E004175A
:103E400011F00C94281FAC81BD818C91885F8C93FC
:103E5000AC81BD810C91003018F011F00C94321F30
:103E60000C948B1F85E090E00E940A2F80E0AA81CD
:103E7000BB818C930027BB27A0E38C9180FB0EF4C1
:103E800001E040E0041711F00C944A1F81E0AA8180
:103E9000BB818C930027BB27A0E38C9181FB0EF4A0
:103EA00001E040E0041711F00C945B1FAA81BB8174
:103EB0008C918E5F8C930027BB27A9E38C9185FBA7
:103EC0000EF401E040E0041711F00C946C1FAA817D
:103ED000BB818C918C5F8C930027BB27A9E38C91CD
:103EE00084FB0EF401E040E0041711F00C947D1FF8
:103EF000AA81BB818C91885F8C93AA81BB814C91F4
:103F0000AC81BD810C91041711F40C948B1F80E0DF
:103F1000AC81BD818C93AC81BD810C91033011F0DB
:103F20000C94981F82E0AC81BD818C930C94CE1FC1
:103F3000AC81BD810C91043081E008F480E08F9366
:103F4000AC81BD810C91073081E010F009F080E078
:103F50009F918923882311F40C94B41F83E0AC81D2
:103F6000BD818C930C94CE1FAC81BD810C91083027
:103F700081E008F480E08F93AC81BD810C910F301B
:103F800081E010F009F080E09F918923882311F4EB
:103F90000C94CE1F84E0AC81BD818C9381E081BB09
:103FA0009198539A549AAC81BD818C91AE81BF8116
:103FB0008C9384E0481A8827580A2696089581E051
:103FC0000E94192F81E00E94192FAC81BD818C9134
:103FD000A881B9818C930E94FA0E88EC90E00E942F
:103FE0000A2F5A924A9281E0A42DB52D8C9381E03C
:103FF0000E94A52D0E94152B229681E00E94A12DE2
:10400000A895E9E6F0E0FA93EA930E94501E229602
:104010008AE090E00E940A2F00916900003011F0C0
:104020000C94002086E990E00E940A2F5A924A924E
:1040300080E0A42DB52D8C9381E00E94A52D0E94D7
:10404000152B229681E00E94A12D84E690E00E942B
:104050000A2F5A924A9280E0A42DB52D8C9381E0CC
:104060000E94A52D0E94152B229681E00E94A12D71
:10407000A895E9E6F0E0FA93EA930E94501E229692
:104080000E94FC0E5A924A9281E0A42DB52D8C9389
:1040900081E00E94A52D0E94152B229681E00E94AE
:1040A000A12D84E690E00E940A2F5A924A9280E065
:1040B000A42DB52D8C9381E00E94A52D0E94152B77
:1040C000229681E00E94A12D8AE090E00E940A2FB2
:1040D0005A924A9280E0A42DB52D8C9381E00E94E3
:1040E000A52D0E94152B229681E00E94A12D0E94F1
:1040F000FA0E86E990E00E940A2F009169000030D4
:1041000018F011F00C9486200C94382088E790E089
:104110000E940A2F5A924A9281E0A42DB52D8C93C9
:1041200081E00E94A52D0E94A721229681E00E9495
:10413000A12DA881B9810C91023011F00C94E020DE
:1041400000916900013011F00C94AB2081E0809364
:10415000C3000C94D920023011F00C94C32080E0ED
:104160008093C3005A924A9281E0A42DB52D8C937E
:1041700081E00E94A52D0E94A721229681E00E9445
:10418000A12D0C94D920033011F00C94D92083E098
:104190008093C3005A924A9282E0A42DB52D8C934D
:1041A00081E00E94A52D0E94A721229681E00E9415
:1041B000A12DEEE0F0E0A3ECB0E07BE70E9404303C
:1041C000A881B9810C91033011F00C941321009156
:1041D0006900013011F00C94F420A4ECB0E08C9153
:1041E00081608C930C940C21023011F00C940C2102
:1041F000A4ECB0E08C918E7F8C935A924A9281E02D
:10420000A42DB52D8C9381E00E94A52D0E94A7219D
:10421000229681E00E94A12DEFE0F0E0A4ECB0E056
:104220007BE70E940430A881B9810C91013011F024
:104230000C94652100916900013011F00C942C213F
:10424000A4ECB0E08C9182608C93A4ECB0E08C91F3
:104250008B7F8C930C945E21023011F00C944621DC
:10426000A4ECB0E08C91897F8C935A924A9281E0C1
:10427000A42DB52D8C9381E00E94A52D0E94A7212D
:10428000229681E00E94A12D0C945E21033011F052
:104290000C945E21A4ECB0E08C9186608C935A92D1
:1042A0004A9282E0A42DB52D8C9381E00E94A52D29
:1042B0000E94A721229681E00E94A12DEFE0F0E06C
:1042C000A4ECB0E07BE70E9404300E94FE0EA895AB
:1042D000E9E6F0E0FA93EA930E94501E229685E008
:1042E00090E00E940A2F00916900003011F00C94B8
:1042F000672186E990E00E940A2F5A924A9280E054
:10430000A42DB52D8C9381E00E94A52D0E94152B24
:10431000229681E00E94A12D86E990E00E940A2F5A
:104320005A924A9280E0A42DB52D8C9381E00E9490
:10433000A52D0E94152B229681E00E94A12D0E949E
:10434000FC0E82E0481A8827580A2496089581E0D6
:104350000E94192F81E0A881B9818C93AA81BB8129
:104360004C91A881B9810C91041718F011F00C94AC
:10437000D4215A924A9282E0A42DB52D8C9381E0EB
:104380000E94A52D0E94152B229681E00E94A12D4E
:104390008DE790E00E940A2FA881B9818C918F5FF0
:1043A0008C9311F00C94AE2181E0481A8827580AAA
:1043B0002296089581E00E94192F81E0A881B98199
:1043C0008C93A881B9810C91063018F011F00C94EF
:1043D000FD210E94FA0E8FE090E00E940A2F0E94B9
:1043E000FC0E84E690E00E940A2FA881B9818C918E
:1043F0008F5F8C9311F00C94E12181E0481A88279B
:10440000580A2296089580E08093C00080E080934F
:10441000C1000E94F62EC39A88EC90E00E940A2FF9
:1044200081B5886081BD0E9468295A924A9281E0D4
:10443000A42DB52D8C9381E00E94A52D5A924A920D
:104440008091C000A42DB52D8C9381E00E94A52DF4
:104450005A924A928091C100A42DB52D8C9381E08F
:104460000E94A52D0E94B429269683E00E94A12DCA
:1044700081B5886181BD877F81BD84E690E00E941F
:104480000A2FFF27E0E1FA93EA935A924A928BE0CF
:10449000A42DB52D8C9381E00E94A52D0E94AB2CFC
:1044A000249681E00E94A12D013051E0150711F002
:1044B0000C9473225A924A92ACEBB0E08D919C918D
:1044C000A42DB52D8D939C9382E00E94A52D0E9472
:1044D000BB2A229682E00E94A12DE6E0F1E60E942E
:1044E000512E0E945D2E5A924A9282E3A42DB52D40
:1044F0008C9381E00E94A52D5A924A928091C0002F
:10450000A42DB52D8C9381E00E94A52D5A924A923C
:104510008091C100A42DB52D8C9381E00E94A52D22
:104520000E94B429269683E00E94A12DC29AD89AAF
:1045300082E390E00E940A2F089581E00E94192FE3
:1045400081E00E94192F8FEFAA81BB818C9380E0BC
:10455000A881B9818C93A881B9810C91073018F09A
:1045600011F00C94C02291E0AA81BB810E94EC2E34
:10457000A881B9818C918F5F8C9311F00C94AB2240
:1045800082E0481A8827580A2496089581E00E94FC
:10459000192F81E00E94192F81E00E94192F82E0DB
:1045A0000E94192F82E00E94192F8FEFAA85BB85E8
:1045B0008C9381E0A885B9858C93A885B9850C91E9
:1045C000003418F011F00C94EF220E949D22A8856F
:1045D000B9858C918F5F8C9311F00C94DD22C49877
:1045E00081E0A885B9858C93A885B9850C910034A4
:1045F00018F011F00C9406230E949D22A885B9851D
:104600008C918F5F8C9311F00C94F4228AE090E0EF
:104610000E940A2FA895EE81FF81FA93EA935A929D
:104620004A9280E4A42DB52D8C9381E00E94A52DA3
:104630005A924A9200E010E020E030E0A42DB52D1F
:104640000D931D932D933C9384E00E94A52D0E9411
:10465000D728269685E00E94A12DAE81BF810C91BE
:10466000013011F40C943D23C49AEAE0F1E60E9473
:10467000512E0E945D2E0C94F42581E0AA85BB8505
:104680008C93A89580E090E0A881B9818D939C934C
:10469000EE81FF81FA93EA935A924A9281E4A42D23
:1046A000B52D8C9381E00E94A52D5A924A9200E08C
:1046B00010E020E030E0A42DB52D0D931D932D9337
:1046C0003C9384E00E94A52D0E94D728269685E081
:1046D0000E94A12DA881B9810E94B82DAE81BF8111
:1046E0000C91003081E009F080E08F93A881B981BE
:1046F0000D911C91003050E0150781E009F080E039
:104700009F91892B882311F40C944823C49AA88183
:10471000B9810D911C91003050E0150711F00C94F7
:104720009923E2E1F1E60E94512E0E945D2E0C9445
:10473000F425A89584E690E00E940A2FA895C498D5
:1047400081E090E00E940A2FEE81FF81FA93EA93C4
:104750005A924A9280E5A42DB52D8C9381E00E9457
:10476000A52D5A924A9201E010E020E030E0A42DFD
:10477000B52D0D931D932D933C9384E00E94A52DA0
:104780000E94D728269685E00E94A12D85E090E022
:104790000E940A2FC49A8AE090E00E940A2FA895EE
:1047A00000E010E020E030E0AAE7B0E00D931D93B8
:1047B0002D933C9300E010E020E030E0A3EDB0E06A
:1047C0000D931D932D933C930E94FA2500E010E079
:1047D00020E030E0A3EDB0E00D931D932D933C93CA
:1047E0000027A1EDB0E08C9186FB0EF401E041E0E2
:1047F000041711F00C94FE230C94F425A895009155
:10480000E800023011F40C94922480919E0280936F
:104810007E00A5EAB2E00D91112740E051E00E9430
:10482000242EAA81BB810D931C93AA81BB810D917B
:104830001C91A4EAB2E04D915527040F151FAA81DF
:10484000BB810D931C93AA81BB810D911C912227E2
:10485000332740E050E061E070E00E946A2EAAE752
:10486000B0E00D931D932D933D93A3EAB2E00D911B
:10487000112740E051E00E94242EAA81BB810D93B4
:104880001C93AA81BB810D911C91A2EAB2E04D91CB
:104890005527040F151FAA81BB810D931C93AAE70E
:1048A000B0E00D911D912D913C91AA81BB814D915C
:1048B0005C91662777270E94712FAAE7B0E00D93DD
:1048C0001D932D933D9300917E000C3011F00C94BC
:1048D0006C248BE080937E0000917E000E3011F0FE
:1048E0000C9475248BE080937E0000917E000F3045
:1048F00011F00C947E248BE080937E00AAE7B0E058
:104900000D911D912D913C91A3EDB0E00D931D9360
:104910002D933C930E94FA25A3EDB0E00E94C42D94
:104920000C94E62400911201063411F00C94BC247E
:1049300084E080937E0087E3A885B9858C93A88561
:10494000B9850C910C3318F011F00C94BA24A88599
:10495000B985AD90BB24ABEDB0E0AA0DBB1D8C9129
:104960000E94602EA885B9858C918F5F8C9311F081
:104970000C949F240E945D2E00912E01063411F0AC
:104980000C94E6248BE080937E0083E5A885B985AE
:104990008C93A885B9850C91073518F011F00C940B
:1049A000E424A885B985AD90BB24ABEDB0E0AA0D99
:1049B000BB1D8C910E94602EA885B9858C918F5F5C
:1049C0008C9311F00C94C9240E945D2EECE1F1E669
:1049D0000E94512EA8E6B7E0EEE7F0E00E949D2F7E
:1049E0000E94492E0E945D2EEEE2F1E60E94512EB9
:1049F000A8E6B7E0EAE7F0E00E94912F0E94492E76
:104A00000E945D2E84E0A885B9858C93A885B98520
:104A10000C910B3018F011F00C942125A885B98564
:104A2000AD90BB24ABEDB0E0AA0DBB1D8C910E94F4
:104A3000602EA885B9858C918F5F8C9311F00C94B2
:104A400006250E945D2E8091E90080936F00E0E4CE
:104A5000F1E60E94512EA8E6B7E0EFE6F0E00E94F2
:104A60009D2F0E94492E0E945D2E00916F00003004
:104A700011F00C943D250C94F42500916F00003446
:104A800018F011F00C9446250C9448250C94F4254C
:104A90008091EA00AE81BF818C938091EB00AC8164
:104AA000BD818C93AC81BD819C91AE81BF818C9185
:104AB000ADE6B0E08D939C938091F200AE81BF8112
:104AC0008C938091F300AC81BD818C93AC81BD81CE
:104AD0009C91AE81BF818C91A0E7B0E08D939C93B7
:104AE000A0E7B0E00D911C91003050E0150711F0E7
:104AF0000C94902580910001AE81BF818C938091B0
:104B00000101AC81BD818C93AC81BD819C91AE8152
:104B1000BF818C91A0E7B0E08D939C930C9490257D
:104B2000A0E7B0E00D911C91003050E0150711F0A6
:104B30000C949C250C94F42502E010E020E030E079
:104B4000A0E7B0E04D915C91662777270E946A2E1E
:104B5000A2E7B0E00D931D932D933D93A2E7B0E043
:104B60000D911D912D913C91ADE6B0E04D915C9180
:104B7000662777270E94712FA2E7B0E00D931D935F
:104B80002D933D93A2E7B0E00D911D912D913C91A5
:104B9000A3EDB0E04D915D916D917C910E94712FDC
:104BA000A2E7B0E00D931D932D933D93E0E5F1E670
:104BB0000E94512EA8E6B7E0E2E7F0E00E94912FB4
:104BC0000E94492E0E945D2EA2E7B0E00D911D913A
:104BD0002D913C91A3EDB0E00D931D932D933C934B
:104BE00080E0AA85BB858C9387E0481A8827580AFD
:104BF0002A96089581E00E94192F81E00E94192FC2
:104C000082E00E94192F82E00E94192F8FEFAE815F
:104C1000BF818C9391E0AE81BF810E94EC2E91E028
:104C2000AE81BF810E94EC2E91E0AE81BF810E94D7
:104C3000EC2E91E0AE81BF810E94EC2E91E0AE811E
:104C4000BF810E94EC2E91E0AE81BF810E94EC2ECC
:104C500091E0AE81BF810E94EC2E91E0AE81BF81D8
:104C60000E94EC2E91E0AE81BF810E94EC2E91E07B
:104C7000AE81BF810E94EC2E91E0AE81BF810E9487
:104C8000EC2E91E0AE81BF810E94EC2E91E0AE81CE
:104C9000BF810E94EC2E91E0AE81BF810E94EC2E7C
:104CA00091E0AE81BF810E94EC2E91E0AE81BF8188
:104CB0000E94EC2EC49880E090E0A881B9818D9389
:104CC0009C938FEF0E94FD2E0E94FF2E0E94FE2ECD
:104CD000AE81BF818C93A881B9810E94B82DAE812D
:104CE000BF810C91003081E009F480E08F93A881AE
:104CF000B9810D911C91003050E0150781E009F059
:104D000080E09F91892B882311F40C946126A8815F
:104D1000B9810D911C91003050E0150711F00C94F1
:104D20009E26E8E5F1E60E94512E0E945D2E7091CC
:104D3000D10070647093D1000C94EB27EE81FF8159
:104D4000FA93EA935A924A9281E5A42DB52D8C9359
:104D500081E00E94A52D5A924A92A3EDB0E00D91F8
:104D60001D912D913C91A42DB52D0D931D932D9347
:104D70003C9384E00E94A52D0E94D728269685E0CA
:104D80000E94A12D0027A1EDB0E08C9186FB0EF4CE
:104D900001E041E0041711F00C94DE26E6E6F1E6AE
:104DA0000E94512EA8E6B7E0E3EDF0E00E94912FBB
:104DB0000E94492E0E945D2E0C94EB27A895AE818F
:104DC000BF810C91003011F00C94292780E090E015
:104DD000A881B9818D939C938FEF0E94FD2E0E9434
:104DE000FF2E0E94FE2EAE81BF818C93A881B981D7
:104DF0000E94B82DAE81BF810C91003081E009F492
:104E000080E08F93A881B9810D911C91003050E012
:104E1000150781E009F080E09F91892B882311F428
:104E20000C94EC26A881B9810D911C91003050E0C2
:104E3000150711F00C942927E0E8F1E60E94512EA5
:104E40000E945D2E7091D10070647093D1000C941B
:104E5000EB27AE81BF810C910F3F11F00C947327AB
:104E600080E090E0A881B9818D939C938FEF0E94A0
:104E7000FD2E0E94FF2E0E94FE2EAE81BF818C93DC
:104E8000A881B9810E94B82DAE81BF810C910F3FDE
:104E900081E009F480E08F93A881B9810D911C9184
:104EA000003050E0150781E009F080E09F91892BE8
:104EB000882311F40C943627A881B9810D911C9197
:104EC000003050E0150711F00C947327EEE8F1E67E
:104ED0000E94512E0E945D2E7091D10070647093DB
:104EE000D1000C94EB27AE81BF810C910E3F11F4E1
:104EF0000C949027ECE9F1E60E94512EA8E6B7E069
:104F0000EE81FF810E949D2F0E94492E0E945D2EFE
:104F1000C49A7091D10070647093D1000C94EB2707
:104F200080E090E0AA81BB818D939C9380E0AE816C
:104F3000BF818C93AE81BF810C910F3F18F011F0AF
:104F40000C94D227AA81BB810E94B82D8FEF0E94BA
:104F5000FD2E0E94FF2E0E94FE2EAA81BB81AD90E5
:104F6000BC90ABEDB0E0AA0DBB1D8C93AA81BB81B8
:104F70000E94B82D8FEF0E94FD2E0E94FF2E0E94EE
:104F8000FE2EAA81BB81AD90BC90ABEDB0E0AA0D26
:104F9000BB1D8C93AE81BF818C918F5F8C9311F080
:104FA0000C949A278FEF0E94FD2E0E94FF2E0E94E4
:104FB000FE2EAE81BF818C938FEF0E94FD2E0E944A
:104FC000FF2E0E94FE2EAE81BF818C93C49AA3ED6A
:104FD000B0E00E94A92D86E0481A8827580A289632
:104FE000089582E00E94192F81E00E94192F80E02D
:104FF000AE81BF818C930E949D22C49880E090E096
:10500000AA81BB818D939C938FEF0E94FD2E0E94FD
:10501000FF2E0E94FE2EA881B9818C93AA81BB81AC
:105020000E94B82DA881B9810C91003081E009F46B
:1050300080E08F93AA81BB810D911C91003050E0DC
:10504000150781E009F080E09F91892B882311F4F6
:105050000C940428AA81BB810D911C91003050E072
:10506000150711F00C944128E8E5F1E60E94512E55
:105070000E945D2E7091D10070647093D1000C94E9
:10508000D128E881F981FA93EA935A924A9281E50C
:10509000A42DB52D8C9381E00E94A52D5A924A92A1
:1050A000AA85BB850D911D912D913C91A42DB52D07
:1050B0000D931D932D933C9384E00E94A52D0E9497
:1050C000D728269685E00E94A12DA881B9810C9150
:1050D000003011F00C94982880E090E0AA81BB8108
:1050E0008D939C938FEF0E94FD2E0E94FF2E0E94B5
:1050F000FE2EA881B9818C93AA81BB810E94B82D14
:10510000A881B9810C91003081E009F480E08F938F
:10511000AA81BB810D911C91003050E0150781E000
:1051200009F080E09F91892B882311F40C94722858
:10513000A881B9810C910F3F11F00C94CB2880E02D
:1051400090E0AA81BB818D939C938FEF0E94FD2EEE
:105150000E94FF2E0E94FE2EA881B9818C93AA8105
:10516000BB810E94B82DA881B9810C910F3F81E0CD
:1051700009F480E08F93AA81BB810D911C910030CE
:1051800050E0150781E009F080E09F91892B88238A
:1051900011F40C94A528A881B9818C91AE81BF81AE
:1051A0008C9383E0481A8827580A2496089584E04F
:1051B0000E94192F81E00E94192F82E00E94192F6E
:1051C0008FEFAA81BB818C9391E0AA81BB810E9461
:1051D000EC2E91E0A885B9850E94EC2EAE81BF81AE
:1051E0000D911D912D913C9140E052E060E070E006
:1051F0000E946A2EAC81BD810D931D932D933D932A
:10520000AC81BD818F9314968E910E945D298E9101
:105210000E945D298E910E945D298E910E945D29D8
:1052200085E90E945D298F9180E090E0A881B98195
:105230008D939C938FEF0E94FD2E0E94FF2E0E9463
:10524000FE2EAA81BB818C93A881B9810E94B82DC2
:10525000AA81BB810C910F3F81E009F480E08F931C
:10526000A881B9810D911C91003050E0150781E0B3
:1052700009F080E09F91892B882311F40C941A295E
:10528000A881B9810D911C91003050E0150711F0F3
:105290000C945529EAEAF1E60E94512E0E945D2EF7
:1052A0007091D10070647093D100AA81BB818C9100
:1052B000AA85BB858C930C9462298FB9779BFECF0E
:1052C0008FB1089587E0481A8827580A26960895CE
:1052D0005A924A9284E298E0A42DB52D8D939C9326
:1052E00082E00E94A52D5A924A9280E0A42DB52D0D
:1052F0008C9381E00E94A52D0E94502C249683E07F
:105300000E94A12DEF93FF93ECE8F1E00E94DE2EC6
:10531000FF91EF91BB27A0E38C9182FBDEF789E13F
:1053200090E00E940A2F5A924A9280E298E0A42DBF
:10533000B52D8D939C9382E00E94A52D5A924A929E
:1053400080E0A42DB52D8C9381E00E94A52D0E94B4
:10535000502C249683E00E94A12D89E190E00E94C8
:105360000A2F0E94D82A089582E00E94192F82E015
:105370000E94192F82E00E94192FA885B9850C91EF
:10538000003081E009F080E08F93AE81BF810C9105
:10539000003081E009F080E09F918923882311F497
:1053A0000C94E429AA85BB858C91AA81BB818D933D
:1053B00088278C93AA85BB858C91A881B9818D9310
:1053C00088278C930C94262AAA85BB850D911127DA
:1053D000A885B9854D915527040F151FAA81BB815A
:1053E0000D931C93AA81BB810D911C910F3F50E03E
:1053F000150718F011F00C94FF290C94052A8FEF73
:1054000090E0AA81BB818D939C93AA85BB850D9169
:105410001127AE81BF814D915527040F151FA8811B
:10542000B9810D931C93A881B9810D911C910F3FF7
:1054300050E0150718F011F00C94202A0C94262A3D
:105440008FEF90E0A881B9818D939C9300E011E0EB
:10545000AA81BB814D915C910E94242EAC81BD81BB
:105460000D931C93AC81BD810D911C91A881B981D4
:105470004D915C91040F151FAC81BD810D931C9360
:105480005A924A92AE81BF818D919C91A42DB52DE7
:105490008D939C9382E00E94A52D5A924A928BE0B4
:1054A000A42DB52D8C9381E00E94A52D0E94502C37
:1054B000249683E00E94A12D5A924A9280E298E0BD
:1054C000A42DB52D8D939C9382E00E94A52D5A9218
:1054D0004A9280E0A42DB52D8C9381E00E94A52DE9
:1054E0000E94502C249683E00E94A12D86E0481A49
:1054F0008827580A2696089582E00E94192F00E115
:1055000010E0AC81BD814D9155270E94242EA881C9
:10551000B9810D931C93A881B9810D911C91AA8129
:10552000BB814D915527040F151FA881B9810D939B
:105530001C935A924A92AA81BB818D919C91A42D71
:10554000B52D8D939C9382E00E94A52D5A924A928C
:1055500082E0A42DB52D8C9381E00E94A52D0E94A0
:10556000502C249683E00E94A12D82E0481A8827BF
:10557000580A229608955A924A92AA81BB818D9127
:105580009C91A42DB52D8D939C9382E00E94A52D16
:105590005A924A9283E0A42DB52D8C9381E00E940B
:1055A000A52D0E94502C249683E00E94A12D0895E1
:1055B00081E00E94192F81E00E94192FC49AD89887
:1055C000C29880E0A881B9818C9380E0AA81BB81D8
:1055D0008C93AA81BB810C910F3118F011F00C94BF
:1055E0000D2B91E0A881B9810E94EC2E91E0A88159
:1055F000B9810E94EC2E91E0A881B9810E94EC2E25
:1056000091E0A881B9810E94EC2EAA81BB818C9186
:105610008F5F8C9311F00C94E92AC29AD89A82E099
:10562000481A8827580A2496089581E00E94192F65
:105630005A924A9280E298E0A42DB52D8D939C93C6
:1056400082E00E94A52D5A924A9280E0A42DB52DA9
:105650008C9381E00E94A52D0E94502C249683E01B
:105660000E94A12DAA81BB810C91003011F00C94F5
:10567000482B5A924A9280E0A42DB52D8C9381E05C
:105680000E94A52D0E94C22B229681E00E94A12D8E
:10569000AA81BB810C91013011F00C945E2B5A92BF
:1056A0004A9285E6A42DB52D8C9381E00E94A52D0C
:1056B0000E94C22B229681E00E94A12DAA81BB816B
:1056C0000C91023011F00C948B2B5A924A9283E683
:1056D000A42DB52D8C9381E00E94A52D0E94C22B94
:1056E000229681E00E94A12D88EC90E00E940A2F72
:1056F0005A924A9280E0A42DB52D8C9381E00E94AD
:10570000A52D0E94C22B229681E00E94A12D82E34A
:1057100090E00E940A2FAA81BB810C91033011F006
:105720000C94B42B5A924A9282E6A42DB52D8C93F8
:1057300081E00E94A52D0E94C22B229681E00E944A
:10574000A12D80E991E00E940A2F5A924A9280E0AE
:10575000A42DB52D8C9381E00E94A52D0E94C22B13
:10576000229681E00E94A12D8AE090E00E940A2FFB
:105770008AE090E00E940A2F81E0481A8827580AA0
:105780002296089581E00E94192FC49AD898C29851
:10579000AA81BB810C91003018F011F00C94D22B2F
:1057A0000C940C2C83E5A881B9818C9391E0A8819D
:1057B000B9810E94EC2E8FEEA881B9818C9391E083
:1057C000A881B9810E94EC2E8EE6A881B9818C93C4
:1057D00091E0A881B9810E94EC2E91E0AA81BB8161
:1057E0000E94EC2E80E0A881B9818C9391E0A88181
:1057F000B9810E94EC2E91E0A881B9810E94EC2E23
:1058000091E0A881B9810E94EC2E91E0A881B98134
:105810000E94EC2E0C94482C85E4A881B9818C93CD
:1058200091E0A881B9810E94EC2E88E7A881B98116
:105830008C9391E0A881B9810E94EC2E89E6A88121
:10584000B9818C9391E0A881B9810E94EC2E84E704
:10585000A881B9818C9391E0A881B9810E94EC2E36
:1058600080E0A881B9818C9391E0A881B9810E94E0
:10587000EC2E91E0A881B9810E94EC2E91E0A881E4
:10588000B9810E94EC2E91E0A881B9810E94EC2E92
:10589000C29AD89A81E0481A8827580A2296089511
:1058A00081E00E94192FC29AD8985A924A9282E0B7
:1058B000A42DB52D8C9381E00E94A52D0E94052D6D
:1058C000229681E00E94A12D5A924A92AC81BD811C
:1058D0008C91A42DB52D8C9381E00E94A52D0E9462
:1058E000052D229681E00E94A12DAC81BD811196EB
:1058F0008C91A881B9818C935A924A92AA81BB81DA
:105900008C91A42DB52D8C9381E00E94A52D0E9431
:10591000052D229681E00E94A12DAC81BD818C9144
:10592000A881B9818C935A924A92AA81BB818C91A9
:10593000A42DB52D8C9381E00E94A52D0E94052DEC
:10594000229681E00E94A12DD89A81E0481A8827EA
:10595000580A2296089581E00E94192F81E00E9442
:10596000192F82E00E94192FC29AD8985A924A920F
:1059700083E0A42DB52D8C9381E00E94A52D0E947B
:10598000052D229681E00E94A12D5A924A92A88567
:10599000B9858C91A42DB52D8C9381E00E94A52D05
:1059A0000E94052D229681E00E94A12DEC81FD81AF
:1059B000FA93EA930E940B2D2296EA81FB81FA93D7
:1059C000EA930E940B2D2296D89AAC81BD810D914D
:1059D000112740E051E00E94242EA881B9810D9347
:1059E0001C93A881B9810D911C91AA81BB814D9115
:1059F0005527040F151FA885B9850D931C9384E0C6
:105A0000481A8827580A2696089591E0A881B981F6
:105A10000E94EC2E089581E00E94192F91E0A88148
:105A2000B9810E94E12EA881B9818C91AA81BB81A4
:105A30008C9381E0481A8827580A2296089582E0BC
:105A40000E94192F81E00E94192FC49ABB27A0E35E
:105A50008C9182FBDEF7C298AC81BD810D911C91C7
:105A6000003052E0150711F00C946E2D81E090E0AB
:105A7000AA81BB818D939C9380E0A881B9818C938E
:105A8000A881B9810C910F3018F011F00C946C2D95
:105A9000BB27A0E38C9182FBDEF790E2AA81BB8159
:105AA000AD90BC90ABEDB0E0AA0DBB1D0E94EC2EFA
:105AB000AA81BB810D911C9140E250E0040F151F9B
:105AC000AA81BB810D931C93A881B9818C918F5FB2
:105AD0008C9311F00C94402D0C949A2D81E090E061
:105AE000AA81BB818D939C93AC81BD814D915C91CA
:105AF000AA81BB810D911C910417150718F011F0B4
:105B00000C949A2DBB27A0E38C9182FBDEF7C29AFE
:105B100091E0AA81BB81AD90BC90ABEDB0E0AA0D45
:105B2000BB1D0E94EC2EAA81BB810E94B82D11F0F2
:105B30000C94742DC29A83E0481A8827580A249638
:105B40000895481A8827580A0895480E8827581E2D
:105B500008950D911D912D913C9181E0080F8827AA
:105B6000181F281F381F3C932E931E930E930895E1
:105B7000ED91FC913196FC93EE930895ED91FC919B
:105B80003197FC93EE9308950D911D912D913C91C9
:105B900001501040204030403C932E931E930E93B2
:105BA00008954091DD025091DE020DE815E30E9458
:105BB000E52D49E156E3040F151F0093DD02109314
:105BC000DE02498158810C940A2E08D03DD000FC99
:105BD00010D0089503D01ED001F8F9CF0024E89426
:105BE00057FF02C009D0689400F80BD010F80124C8
:105BF000089502D009D00895509540954F5F5F4FAA
:105C00000895E89417FF0895009510950F5F1F4FB2
:105C100068940895352F242FE894452B11F4689447
:105C20000895512F402F0027112780E1440F551F61
:105C3000001F111F021B130B416018F4020F131FEA
:105C40004E7F8A9599F708950F92049F202C312C4E
:105C5000419F300C509F030C022D102D0F90089582
:105C6000C8950D9231960020D9F708958F938D91A4
:105C70008823E9F711978F91089581E05F9B88272A
:105C8000089588275F9B089500C05F9BFECF8CB16D
:105C90000895A8E6B7E08D91882311F011D0FBCFCD
:105CA00008950E941F2F802D11F00AD0FACF089579
:105CB0008D9106D03A95E1F708958DE001D08AE004
:105CC0005D9BFECF8CB9089588EE93E0A3D0319709
:105CD000D9F7089550D00AD000FC05D008954BD0D4
:105CE00020D001F8F9CF52D05AD00895842F952FA3
:105CF000A62FB72F4427552766277727F1E28894E8
:105D000009C020F4480F591F6A1F7B1F76956795BD
:105D1000579547953795279517950795FA9589F7DC
:105D20000895842F952FA62FB72FE894452B462B47
:105D3000472B11F468940895402F512F622F732F31
:105D40000027112722273327F0E2440F551F661F33
:105D5000771F001F111F221F331F081B190B2A0B4F
:105D60003B0B416028F4080F191F2A1F3B1F4E7F71
:105D7000FA9559F708950024E89477FF02C006D0F9
:105D8000689400F809D010F80124089512D04F5FEC
:105D90005F4F6F4F7F4F0895E89437FF0895009548
:105DA0001095209530950F5F1F4F2F4F3F4F6894F0
:105DB0000895409550956095709508953197F1F745
:105DC00008950E94FD2E8C910E94FF2E8D939A952E
:105DD000D1F70E94FE2E08950E94FD2E8D910E9403
:105DE000FF2E9A95D9F70E94FE2E0895BF9ABE986D
:105DF000C69ABD9A80E58DB90895089508958FB922
:105E0000779BFECF8FB10895689462F80895E89467
:105E100062F80895EF93FF93EE27E82BE92B31F01A
:105E2000E0EDF7E03197F1F70197D1F7FF91EF91AE
:105E300008955A924A92480E8827581E0895C89588
:105E4000319600200895819104D08D938823D9F74D
:105E50000895813618F08B3708F48F7D089580E31C
:105E60000EF4839508952E2E3F2E992781918D3221
:105E700009F093958823D1F79A95E22DF32D1123FC
:105E800061F0091718F011F0101B01C0191B28F060
:105E900021F080E28D931A95E9F780818D3219F413
:105EA0008D93319604C0222311F08BE28D93091754
:105EB00038F031F0091B21F080E38D930A95E9F762
:105EC00081918D938823E1F7332351F0EA2FFB2F43
:105ED000319633958E9182933A95E1F78EE28C93C9
:105EE0000895040F151F261F371F0895041B150B57
:105EF000260B370B08950417150726073707089553
:105F0000000F111F221F331F089500951095209533
:105F100030950F5F1F4F2F4F3F4F08950191108114
:105F20000EC001911191219130810BC0019110811E
:105F300017FF05C03FEF2FEF04C000811127222774
:105F4000332737FF03C0E1DF8DE28D93CF93DF93DB
:105F5000CF92DF92EF92AA24BB24CC24DD24EE243E
:105F600040E2CAE0DD2755E093E38881890F87FD91
:105F70009F7083FD907F891B89935A95A9F7C0DF95
:105F8000AA1CBB1CCC1CDD1CEE1C4A9551F7E894E6
:105F9000EFE0FF2782910ED0EB30E0F71EF068941F
:105FA0008A2D0CD088278D93EF90DF90CF90DF91D2
:105FB000CF910895982F829501D0892F8F70805DA1
:105FC00026F0803309F4089568948D930895882706
:105FD0008D93089581918D938823E1F70895099118
:105FE0009191992351F08A95D9F7319781918D93A9
:105FF0000A9519F08823D1F70895E9CFE199FECFEA
:10600000EEBBFFBB3196089591E001C092E07B3773
:1060100051F47FB7F894F2DF8D918DBBE29AE19A4B
:106020009A95C9F77FBF7727089591E001C092E064
:10603000E5DFE09A8DB38D939A95D1F70895FF939C
:10604000881BF9E0001FFA9511F4FF910895881F4D
:10605000841B18F4840F8894F5CF0894F3CF6894C8
:1060600001C0E894AF93BF938D9116F0919103C056
:106070000E941F2F902D891718F011F48823A1F783
:10608000BF91AF9108954D50335354414D5020521C
:1060900065616C6974792D53797320342E37000053
:1060A00053005000454570726F6D20002C004D4D1F
:1060B0004320696E697420007265747279202E2EF7
:1060C0002E0044535020696E697420004F005A001E
:1060D00059004B005500470052005700410048004E
:1060E00021004E00420058004400450056004D007B
:1060F000540049004C00434F4E46494700002000E1
:10610000442000002E006F6B00004E6F2063617210
:1061100064004261642063617264000050617274C3
:106120006974696F6E2074797065203A000050615F
:1061300072746974696F6E2073746172743A0000CE
:10614000536563742F636C757374657220203A0015
:10615000526F6F74203A000052656164206572725C
:106160006F722031000052656164206572726F7237
:106170002032206F6E20736563746F723A200000C6
:1061800052656164206572726F722033000052653F
:106190006164206572726F72203400005265616420
:1061A000206572726F722035000052656164207440
:0861B000696D656F7574000054
:00000001FF
